:1000000020C03AC039C038C037C036C035C034C04F
:1000100033C032C031C030C02FC02EC02DC02CC064
:100020002BC0BAC1E3C1ECC1E6C1D8C1FCC1FBC160
:10003000FAC1CBC1C5C1F7C1DEC1CCC1CBC1F3C1CF
:10004000EBC111241FBECFE5D2E0DEBFCDBF10E073
:10005000A0E6B0E0E8E8F4E002C005900D92A23618
:10006000B107D9F710E0A2E6B0E001C01D92A536B5
:10007000B107E1F7F9D006C2C3CF80E88ABB8FE1B0
:1000800087BB089590916000981789F098B3987F86
:1000900098BBDF9828B3982F9770922B98BB2BB3FF
:1000A000982F92959078922B9BBB80936000089537
:1000B0001F93CF93DF93EC011091600080E0E2DFAB
:1000C00020E030E003C000002F5F3F4F2C173D07BA
:1000D000D4F3812FD7DFDF91CF911F91089585E071
:1000E000D1DF8FE39DE0A3E081509040A040E1F795
:1000F00000C0000080E0C6DFA7EAB1E61197F1F783
:1001000000C000008AE0BEDF8FE39DE0A3E08150E5
:100110009040A040E1F700C0000080E0B3DF089508
:1001200029B330E02F70307080916200882321F075
:100130008FE090E028273927C9010895EF92FF92B8
:100140000F931F93CF93DF938AE09CDF87EA91E6BA
:100150000197F1F700C0000080E094DFC0E0D0E03C
:1001600003E010E0CE01B80166D1009711F480E001
:1001700089DFD6DF009749F486E084DF2196C83C0A
:10018000D10581F701E010E002C000E010E080E05E
:1001900079DF01301105F1F000E010E0C853DF4FC6
:1001A00083E0E82EF12C0EC0C801B70144D10097BE
:1001B00011F480E067DFB4DF009739F489E062DF93
:1001C0000F5F1F4FC017D1077CF780E05BDF21E096
:1001D00030E002C020E030E0C901DF91CF911F91F3
:1001E0000F91FF90EF9008950F931F93CF93DF939C
:1001F0008AE048DF87EA91E60197F1F700C0000046
:1002000080E040DFC0E0D0E003E010E0CE01B801C4
:1002100012D1009711F480E035DF82DF009719F0EA
:10022000CB30D1059CF480916400813011F489E0D9
:1002300029DF80916400823011F486E023DF21966B
:10024000C83CD10519F7C0E0D0E002C0C1E0D0E061
:1002500080E018DF21E030E02C273D27C901DF9145
:10026000CF911F910F910895BF92CF92DF92EF929D
:10027000FF920F931F93CF93DF9383E294EF019745
:10028000F1F700C00000F9DEA1EEB4E01197F1F73C
:1002900000C0000080E0F6DECD9913C02FE936E8FB
:1002A00041E0215030404040E1F700C0000017DF3E
:1002B0008FE996E8A1E081509040A040E1F700C0AE
:1002C0000000CE9903C081E080936200A3ECB9E006
:1002D0001197F1F700C00000D69AE3ECF9E03197EE
:1002E000F1F700C000008BB390E489278BBB2FE9A6
:1002F00036E841E0215030404040E1F700C00000C6
:100300008BB389278BBB8FE996E8A1E081509040A1
:10031000A040E1F700C0000090E409C08BB389273A
:100320008BBBA3EDB0E31197F1F700C00000CD99AE
:10033000F5CF2FE33DE043E0215030404040E1F76E
:1003400000C00000C0E0D0E000E010E0EE24FF2498
:1003500020E4B22EDD24D39492E0C92E02C0C0E086
:10036000D0E00894E11CF11C30E7E31637E1F30616
:100370002CF08BB38B258BBBEE24FF24E0FC02C05A
:1003800080E080DECDDEE82FF0E0E031F10508F01E
:100390004AC0EF5EFF4F09944EE4C132D40710F01B
:1003A000DE9A46C0219680916400823011F481E08B
:1003B00005C0813011F484E001C085E063DE29C00E
:1003C00085E060DE10926400CACF85E05BDEC092FB
:1003D0006400C5CF84E056DE84E003C086E052DED0
:1003E00086E080936300C092640011C085E04ADE1D
:1003F000D0926400B4CF81E045DED092630005C0A6
:1004000089E040DE89E080936300D0926400C0E020
:10041000D0E000E010E0A5CF0115110509F09FCF55
:10042000E3DE8C019CCF0115110511F485E001C0BC
:1004300080E028DE96CF97FB092E07260AD077FDAD
:1004400004D00CD006D000201AF4709561957F4F2F
:100450000895F6F7909581959F4F0895AA1BBB1BB1
:1004600051E107C0AA1FBB1FA617B70710F0A61BB4
:10047000B70B881F991F5A95A9F780959095BC01D5
:08048000CD010895F894FFCFAF
:02048800FF0073
:00000001FF
